:100000000C9434060C9451060C9451060C94510631
:100010000C9451060C9451060C94F9060C9451065C
:100020000C9451060C9453060C9451060C945106F2
:100030000C9451060C9451060C9451060C945106E4
:100040000C9451060C9451060C9451060C945106D4
:100050000C945106FFFFFFFFFFFFFFFFFFFFFFFFB5
:10006000FFFFFFFFFFFFFFFFFFFFFFFFFFFFFFFFA0
:10007000FFFFFFFFFFFFFFFFFFFFFFFFFFFFFFFF90
:10008000FFFFFFFFFFFFFFFFFFFFFFFFFFFFFFFF80
:10009000FFFFFFFFFFFFFFFFFFFFFFFFFFFFFFFF70
:1000A000FFFFFFFFFFFFFFFFFFFFFFFFFFFFFFFF60
:1000B000FFFFFFFFFFFFFFFFFFFFFFFFFFFFFFFF50
:1000C000FFFFFFFFFFFFFFFFFFFFFFFFFFFFFFFF40
:1000D000FFFFFFFFFFFFFFFFFFFFFFFFFFFFFFFF30
:1000E000FFFFFFFFFFFFFFFFFFFFFFFFFFFFFFFF20
:1000F000FFFFFFFFFFFFFFFFFFFFFFFFFFFFFFFF10
:10010000FFFFFFFFFFFFFFFFFFFFFFFFFFFFFFFFFF
:10011000FFFFFFFFFFFFFFFFFFFFFFFFFFFFFFFFEF
:10012000FFFFFFFFFFFFFFFFFFFFFFFFFFFFFFFFDF
:10013000FFFFFFFFFFFFFFFFFFFFFFFFFFFFFFFFCF
:10014000FFFFFFFFFFFFFFFFFFFFFFFFFFFFFFFFBF
:10015000FFFFFFFFFFFFFFFFFFFFFFFFFFFFFFFFAF
:10016000FFFFFFFFFFFFFFFFFFFFFFFFFFFFFFFF9F
:10017000FFFFFFFFFFFFFFFFFFFFFFFFFFFFFFFF8F
:10018000FFFFFFFFFFFFFFFFFFFFFFFFFFFFFFFF7F
:10019000FFFFFFFFFFFFFFFFFFFFFFFFFFFFFFFF6F
:1001A000FFFFFFFFFFFFFFFFFFFFFFFFFFFFFFFF5F
:1001B000FFFFFFFFFFFFFFFFFFFFFFFFFFFFFFFF4F
:1001C000FFFFFFFFFFFFFFFFFFFFFFFFFFFFFFFF3F
:1001D000FFFFFFFFFFFFFFFFFFFFFFFFFFFFFFFF2F
:1001E000FFEFEFEFEFEFEFEFFFEFFFFFFFD7D7D717
:1001F000FFFFFFFFFFFFFFFFFFEBEB81D7D7D70329
:10020000AFAFFFFFFFEFC7BBBFC7FBBBC7EFFFFF32
:10021000FFBF5DBBF7EFDFBB75FBFFFFFFCFAFAFEE
:10022000DF9F6D6B7789FFFFFFEFEFEFFFFFFFFFB2
:10023000FFFFFFFFFFF7EFEFDFDFDFDFDFEFEFF7BE
:10024000FFDFEFEFF7F7F7F7F7EFEFDFFFFFFF93D2
:10025000C701C793FFFFFFFFFFFFFFEFEFEF01EFC6
:10026000EFEFFFFFFFFFFFFFFFFFFFFFFFEFDFFFEE
:10027000FFFFFFFFFFFF01FFFFFFFFFFFFFFFFFF8C
:10028000FFFFFFFFFFEFFFFFFFFFFDFBF7EFDFBF0C
:100290007FFFFFFFFFC7BBBBBBBBBBBBBBC7FFFF3A
:1002A000FFEF8FEFEFEFEFEFEF83FFFFFFC7BBFB3A
:1002B000FBF7EFDFBF83FFFFFFC7BBFBFBE7FBFBEA
:1002C000BBC7FFFFFFF7E7E7D7D7B783F7E3FFFF2A
:1002D000FF83BFBFBF87FBFBBBC7FFFFFFE7DFBFDE
:1002E000BF87BBBBBBC7FFFFFF83BBFBF7F7EFEFCE
:1002F000DFDFFFFFFFC7BBBBBBC7BBBBBBC7FFFF8E
:10030000FFC7BBBBBBC3FBFBF7CFFFFFFFFFFFFF7D
:10031000EFFFFFFFFFEFFFFFFFFFFFFFEFFFFFFF1D
:10032000FFEFDFFFFFFFFFF7EFDFBFDFEFF7FFFFBD
:10033000FFFFFFFF83FF83FFFFFFFFFFFFFFFFDFE5
:10034000EFF7FBF7EFDFFFFFFFC7BBFBFBF7EFEFBD
:10035000FFEFFFFFFFC3BD6555555563BFC7FFFFE7
:10036000FFCFEFEFD7D7BB83BB11FFFFFF03BDBDAF
:10037000BD83BDBDBD03FFFFFFC3BD7F7F7F7F7F0B
:10038000BDC3FFFFFF07BBBDBDBDBDBDBB07FFFFBD
:10039000FF01BDBFB787B7BFBD01FFFFFF01BDBFF5
:1003A000B787B7BFBF0FFFFFFFC3BD7F7F7F717DE3
:1003B000BDC3FFFFFF11BBBBBB83BBBBBB11FFFFBB
:1003C000FF83EFEFEFEFEFEFEF83FFFFFFC3F7F7F1
:1003D000F7F7F777778FFFFFFF19BBB7B7AF8FB787
:1003E000BB19FFFFFF07DFDFDFDFDFDFDD01FFFF1F
:1003F000FF39BB9393ABABBBBB11FFFFFF31BB9B83
:100400009BABB3B3BB1BFFFFFFC7BB7D7D7D7D7D7A
:10041000BBC7FFFFFF03BDBDBD83BFBFBF0FFFFF56
:10042000FFC7BB7D7D7D7D7DBBC7C9FFFF03BDBD14
:10043000BD83B7B7BB19FFFFFF837D7F7F83FDFDC2
:100440007D83FFFFFF016DEFEFEFEFEFEFC7FFFFE2
:10045000FF11BBBBBBBBBBBBBBC7FFFFFF11BBBB24
:10046000BBD7D7D7EFEFFFFFFF11BBBBBBABABAB2E
:10047000D7D7FFFFFF11BBD7D7EFD7D7BB11FFFFF0
:10048000FF11BBBBD7D7EFEFEFC7FFFFFF017BF734
:10049000F7EFDFDFBD01FFFFFFC7DFDFDFDFDFDFFC
:1004A000DFDFC7FFFFFF7FBFDFEFF7FBFDFFFFFFD2
:1004B000FFC7F7F7F7F7F7F7F7F7C7FFEFD7BBFF78
:1004C000FFFFFFFFFFFFFFFFFFFFFFFFFFFFFFFF3C
:1004D000FFFFFFFFFFDFEFFFFFFFFFFFFFFFFFFF5C
:1004E000FFFFFFFF87FB837B7B85FFFFFF3FBFBFD6
:1004F00083BDBDBDBD03FFFFFFFFFFFF837D7F7F8A
:100500007D83FFFFFFF3FBFB837B7B7B7B81FFFF17
:10051000FFFFFFFF837D017F7D83FFFFFFE7DFDFBD
:1005200087DFDFDFDF87FFFFFFFFFFFF817B7B7B55
:1005300083FBFBC7FF3FBFBFA79BBBBBBB11FFFF3D
:10054000FFEFFFFF8FEFEFEFEF83FFFFFFF7FFFFFF
:1005500087F7F7F7F7F7C7FFFF3FBFBFB3B7AF8F17
:10056000B739FFFFFFCFEFEFEFEFEFEFEF83FFFFC5
:10057000FFFFFFFF17ABABABAB29FFFFFFFFFFFF99
:10058000279BBBBBBB11FFFFFFFFFFFF837D7D7D73
:100590007D83FFFFFFFFFFFF03BDBDBDBD83BF1F09
:1005A000FFFFFFFF817B7B7B7B83FBF1FFFFFFFF77
:1005B00013CDDFDFDF07FFFFFFFFFFFF837D8FF33B
:1005C0007D83FFFFFFFFDFDF87DFDFDFDBE7FFFF8D
:1005D000FFFFFFFF33BBBBBBB3C9FFFFFFFFFFFF45
:1005E00011BBBBD7D7EFFFFFFFFFFFFF11BBABABCB
:1005F000D7D7FFFFFFFFFFFF11BBC7C7BB11FFFF2F
:10060000FFFFFFFF11BBBBD7D7EFEFCFFFFFFFFF10
:100610000377EFDFBB03FFFFFFF3EFEFEFEF9FEF9A
:10062000EFEFEFF3EFEFEFEFEFEFEFEFEFEFEFEFD6
:10063000FF9FEFEFEFEFF3EFEFEFEF9FFFFF9D6D0A
:1006400073FFFFFFFFFFFFFFFFFFC7C7C7C7C7C796
:10065000C7C7C7FFFF016DEFEFE1EEEEEAE9FFFF6D
:10066000F7C0EEEFEFEFEFEFEFC7FFFFFFFFFFFF8A
:10067000FFFFFFFFFFF7EFFFFBF7FFC1EDEFEFEF2E
:10068000EFC7FFFFFFFFFFFFFFFFFFFFFFDBB7FF2E
:10069000FFFFFFFFFFFFFFFFFFABFFFFFFEFEF835A
:1006A000EFEFEFEFEFEFFFFFFFEFEF83EFEFEF8302
:1006B000EFEFFFFFFFFFE3E3E3E3E3E3E3E3E3FF66
:1006C000FFDEADDBF7EFDFAD52EDFFFFFF07B7B7A2
:1006D000B7B1B6B63631FFFFFFFFFFFFFFFBF7EF05
:1006E000F7FBFFFFFF13B7B7B781B6B6B611FFFF31
:1006F000F78CDDDBDBC7DBDBDD8CFFFFFF016DEFA4
:10070000EFE1EEEEEEC6FFFFFF88DDDDDDDDDDDDD6
:10071000DD80F7FFFFDF83DFD3CDDDDDDD8DFDFF86
:10072000FFEFF7FFFFFFFFFFFFFFFFFFFFF7EFFF09
:10073000FFFFFFFFFFFFFFFFFFB7DBFFFFFFFFFF35
:10074000FFFFFFFFFFEDDBFFFFFFFFFFFFFFFFFFEF
:10075000FFFFFFFFE7C3E7FFFFFFFFFFFFFFFFFF15
:10076000FF8FFFFFFFFFFFFFFFFFFFFFFF03FFFF05
:10077000FFFFFFFFFFFFE3E3E3E3E3E3E3E3E3FF85
:10078000FF04AAAEFFFFFFFFFFFFFFFFFFFFFFFF1A
:10079000E7D7D1B6B631FFFFFFFFFFFFFFDFEFF76F
:1007A000EFDFFFFFFFFFFFFF33B781B6B611FFFF9B
:1007B000FFFBF7FF99DBC7DBDB9CFFFFFFDF83DF7E
:1007C000D3CDDDDDDD88FFFFFFFFFFFF99DDDDDD40
:1007D000DDC1F7FFFFFFFFFFFFFFFFFFFFFFFFFF91
:1007E000F780DDDDDDDDE1FDDDE3FFFFFFFFC9F7C4
:1007F00080DDDDDDE1FDDDE3FFE1FBFBFBFBFBBBC2
:10080000BBC7FFFFFFBEC1DDDDDDC1BEFFFFFFFFD8
:10081000FCC0EFEFEFEFEFEFEFC7FFFFFFF7F7F7EA
:10082000F7F7FFF7F7F7F7FFFFE1DDAFB7DBEDF520
:10083000BB87FFFFDDFF80DEDBC3DBDFDE80FFFF8A
:10084000FFE3DDB2AEAEB2DDE3FFFFFFFFE1DEBFEF
:10085000BB83BBBFDEE1FFFFFFFFFFFFFFEEDDBBA2
:10086000DDEEFFFFFFFFFFFFC1FDFFFFFFFFFFFF0B
:10087000FFFFFFFFFFFF80FFFFFFFFFFFFE3DDA69E
:10088000AAA6AADDE3FFFFFFFFC1F7F7F7F7F7F727
:10089000F7C1FFFFFFF7EBF7FFFFFFFFFFFFFFFFD2
:1008A000FFF7F7F780F7F7F7FF80FFFFFFC1F7F7D4
:1008B000F7F7F7F7F7C1FFFFFFF7FFFFC7F7F7F706
:1008C000F7C1FFFFFFFFFDE1EFEFEFEFEFC7FFFF26
:1008D000FFFFFFFFDDDDDDDDDDC3DFFFFFC0858561
:1008E00085C5F5F5F5E4FFFFFFFFFFFFFFFFF7FF0D
:1008F000FFFFFFFFFFDDFFFFC1BE80BFBEC1FFFFE7
:10090000FF39BB9888ABB0B3BB39FFFFFFFFFFFFD8
:10091000C1BE87BFBEC1FFFFFFFFFFFFFFBBDDEE14
:10092000DDBBFFFFFFFBFFFFC3FBFBFBFBFBFBFF95
:10093000FFC1BEBFBFC1FEFEBEC1FFFFFFFFFFFF85
:10094000C1BEC7F9BEC1FFFFFFDBFFFFC7F7F7F767
:10095000F7C1FFFFFFFBF3EBEBDBC3BBBB11FFFFFB
:10096000FF01BDBFBF83BDBDBD03FFFFFF03BDBD15
:10097000BD83BDBDBD03FFFFFF81DDDFDFDFDFDF47
:10098000DF8FFFFFFF01BBBBBBBBBBBBBB017DFF61
:10099000FF01BDBFB787B7BFBD01FFFFFF6DABABA9
:1009A000ABC7ABABAB6DFFFFFF837DFDFDC3FDFDB3
:1009B0007D83FFFFFF39BBB3B3AB9B9BBB11FFFF35
:1009C000E7299BB3B3AB9B9BBB11FFFFFF19BBB7E1
:1009D000B78FB7B7BB19FFFFFF81DBDBDBDBDBDBEF
:1009E0005B11FFFFFF39BB9393ABABBBBB11FFFFA9
:1009F000FF11BBBBBB83BBBBBB11FFFFFFC7BB7DF5
:100A00007D7D7D7DBBC7FFFFFF01BBBBBBBBBBBB10
:100A1000BB11FFFFFF03BDBDBD83BFBFBF0FFFFF06
:100A2000FFC3BD7F7F7F7F7FBDC3FFFFFF016DEFF2
:100A3000EFEFEFEFEFC7FFFFFF11BBBBBBBBC3FB8C
:100A4000BBC7FFFFFFC7EF836D6D6D83EFC7FFFF70
:100A5000FF11BBD7D7EFD7D7BB11FFFFFF11BBBB30
:100A6000BBBBBBBBBB81FDFFFF11BBBBBBBBC3FBA8
:100A7000FBF1FFFFFF29ABABABABABABAB83FFFF36
:100A8000FF29ABABABABABABAB81FDFFFF0F5F5F48
:100A9000C3DDDDDDDD83FFFFFF18BDBD8DB5B5B561
:100AA000B508FFFFFF1FBFBF83BDBDBDBD03FFFF77
:100AB000FF877BFDDDC1DDFD7B87FFFFFF33ADAD34
:100AC000AD8DADADAD33FFFFFF817B7B7B83DBDB8A
:100AD000BB21FFFFFFFFFFFF87FB837B7B85FFFFC2
:100AE000FFFF017FBF837D7D7D83FFFFFFFF8F774A
:100AF00077077B7B7B87FFFFFFFFFFFF877BE79FFE
:100B00007B87FFFFFFFFFFFF817B7B7B83FBBBC7F7
:100B1000FFFFFFFF837D017F7D83FFFFFFFFFFFF5F
:100B20006DABC7ABAB6DFFFFFFFFFFFF837DE3FB4B
:100B30007D83FFFFFFFFFFFF33BBBBBBB3C9FFFFDD
:100B4000FFF7EFFF33BBBBBBB3C9FFFFFFFFFFFFE7
:100B500033B78FB7B739FFFFFFFFFFFFF1EBEBDBD9
:100B6000DB39FFFFFFFFFFFFBB9393ABBB39FFFFF9
:100B7000FFFFFFFF39BB83BBBB11FFFFFFFFFFFF81
:100B8000837D7D7D7D83FFFFFFFFFFFF279BBBBB39
:100B9000BB11FFFFFFFFFFFF03BDBDBDBD83BF1F37
:100BA000FFFFFFFF837D7F7F7D83FFFFFFFFFFFF51
:100BB00017ABABABAB29FFFFFFFFFFFF11BBBBBB0D
:100BC000C3FBBBC7FFFFFFC7EF836D6D6D83EFC72F
:100BD000FFFFFFFF11BBC7C7BB11FFFFFFFFFFFFF9
:100BE00033BBBBBBB3C9FDFFFFFFFFFF11BBBBC3E3
:100BF000FBF1FFFFFFFFFFFF29ABABABAB83FFFFB9
:100C0000FFFFFFFF29ABABABAB81FDFFFFFFFFFF9A
:100C10001F5F43DDDDC3FFFFFFFFFFFF1DBD8DB580
:100C2000B50DFFFFFFFFFFFF1FBF83BDBD03FFFF2C
:100C3000FFFFFFFF837DE1FD7D83FFFFFFFFFFFFE0
:100C400033AD8DADAD33FFFFFFFFFFFFC1BBBBC3B6
:100C5000DB99FFFF53696D706C650053696D706CB3
:100C6000650076312E32000011241FBECFE5D4E09E
:100C7000DEBFCDBF10E0A0E6B0E0EAE1FBE102C0DC
:100C800005900D92A036B107D9F713E0A0E6B0E0C9
:100C900001C01D92A436B107E1F70E94EA0C0C9442
:100CA0008B0D0C9400001F920F920FB60F9211241F
:100CB0002F938F939F93AF93BF93EF93FF93DF9304
:100CC000CF93CDB7DEB7E2E5F0E083EC808380918F
:100CD000660090916700019690936700809366008C
:100CE000809166009091670022E08D30920741F478
:100CF00010926700109266001092620310926800D2
:100D000080916600909167008A30910539F080915A
:100D10006600909167008B30910559F4A2E3B0E032
:100D2000E2E3F0E08081877F8C93E2E3F0E01082E1
:100D30000BC0E2E3F0E084E08083A2E3B0E0E2E312
:100D4000F0E08081877F8C9381E0809363038091C2
:100D50006600909167008D32910580F410926303D4
:100D60000000000000000000000000000000000083
:100D70000000000000000000000026C08091680014
:100D80008F5F8093680080916800883141F4809182
:100D900062038F5F809362031092680015C00000A9
:100DA0000000000000000000000000000000000043
:100DB0000000000000000000000000000000000033
:100DC0000000000000000000A2E3B0E0E2E3F0E079
:100DD000808188608C93CF91DF91FF91EF91BF91DB
:100DE000AF919F918F912F910F900FBE0F901F90F9
:100DF00018951F920F920FB60F9211242F938F9375
:100E00009F93AF93BF93EF93FF93DF93CF9300D064
:100E1000CDB7DEB780916600909167000196909300
:100E2000670080936600809166009091670021E0E2
:100E30008833920741F41092670010926600109276
:100E4000620310926800809166009091670021E033
:100E50008233920708F1809166009091670021E04B
:100E600085339207C8F4A5E3B0E0E5E3F0E08081C4
:100E700081608C938FE08A8301C000008A81815059
:100E80008A838A818823C9F7A5E3B0E0E5E3F0E02F
:100E900080818E7F8C9318C0A5E3B0E0E5E3F0E09D
:100EA00080818E7F8C938EE1898301C000008981CF
:100EB0008150898389818823C9F7A5E3B0E0E5E300
:100EC000F0E0808181608C9381E080936303809166
:100ED0006600909167008832910540F0809166002D
:100EE0009091670021E08731920790F010926303A0
:100EF00000000000000000000000000000000000F2
:100F0000000000000000000000000000000019C008
:100F1000809168008F5F80936800809168008C30BA
:100F200041F4809162038F5F8093620310926800A6
:100F300008C00000000000000000000000000000E9
:100F400000000F900F90CF91DF91FF91EF91BF9133
:100F5000AF919F918F912F910F900FBE0F901F9087
:100F60001895DF93CF93CDB7DEB7A7E3B0E0E7E303
:100F7000F0E0808180688C93A7E3B0E0E7E3F0E0E5
:100F800080818F7B8C93A7E3B0E0E7E3F0E0808182
:100F900080628C93A7E3B0E0E7E3F0E080818061BA
:100FA0008C93EEE2F0E081E08083EDE2F0E080E51A
:100FB0008083CF91DF910895DF93CF93CDB7DEB7D4
:100FC000EAE2F0E01082EBE2F0E01082E0E4F0E030
:100FD00086E88083E9E2F0E083E38083E0E4F0E008
:100FE0001082EAE2F0E080E18083CF91DF91089502
:100FF000DF93CF93CDB7DEB728970FB6F894DEBF57
:101000000FBECDBFE3C1ECE2F0E080818C83809124
:1010100064009091650022E0883F920709F049C181
:1010200084E18B8389E690E09A83898330C1E981EA
:10103000FA81108289819A8101969A838983E98154
:10104000FA81108289819A8101969A838983E98144
:10105000FA81108289819A8101969A838983E98134
:10106000FA81108289819A8101969A838983E98124
:10107000FA81108289819A8101969A838983E98114
:10108000FA81108289819A8101969A838983E98104
:10109000FA81108289819A8101969A838983E981F4
:1010A000FA81108289819A8101969A838983E981E4
:1010B000FA81108289819A8101969A838983E981D4
:1010C000FA81108289819A8101969A838983E981C4
:1010D000FA81108289819A8101969A838983E981B4
:1010E000FA81108289819A8101969A838983E981A4
:1010F000FA81108289819A8101969A838983E98194
:10110000FA81108289819A8101969A838983E98183
:10111000FA81108289819A8101969A838983E98173
:10112000FA81108289819A8101969A838983E98163
:10113000FA81108289819A8101969A838983E98153
:10114000FA81108289819A8101969A838983E98143
:10115000FA81108289819A8101969A838983E98133
:10116000FA81108289819A8101969A838983E98123
:10117000FA81108289819A8101969A838983E98113
:10118000FA81108289819A8101969A838983E98103
:10119000FA81108289819A8101969A838983E981F3
:1011A000FA81108289819A8101969A838983E981E3
:1011B000FA81108289819A8101969A838983E981D3
:1011C000FA81108289819A8101969A838983E981C3
:1011D000FA81108289819A8101969A838983E981B3
:1011E000FA81108289819A8101969A838983E981A3
:1011F000FA81108289819A8101969A838983E98193
:10120000FA81108289819A8101969A838983E98182
:10121000FA81108289819A8101969A838983E98172
:10122000FA81108289819A8101969A838983E98162
:10123000FA81108289819A8101969A838983E98152
:10124000FA81108289819A8101969A838983E98142
:10125000FA81108289819A8101969A838983E98132
:10126000FA81108289819A8101969A838983E98122
:10127000FA81108289819A8101969A838983E98112
:10128000FA81108289819A8101969A8389833B81B0
:1012900038874885442311F051E0588788859B8121
:1012A00091509B83882309F0C2CE10926500109262
:1012B00064008C81282F30E03F832E834E815F8134
:1012C0004930510569F18E819F818D30910509F476
:1012D00043C02E813F812830310509F068C08091DC
:1012E000640090916500009709F470C080916400DB
:1012F00090916500FC01E759FF4F108280916400D6
:1013000090916500019790936500809364008091AF
:10131000640090916500FC01E759FF4F108256C0B0
:101320008091640090916500059632E0883F9307B4
:1013300008F04CC08091640090916500FC01E75971
:10134000FF4F108280916400909165000596909304
:101350006500809364003AC08091640090916500BC
:1013600026E230E0B9010E94770DCB018D838D819B
:10137000833160F58091640090916500FC01E7592C
:10138000FF4F10828D81882F90E09C012F5F3F4F8F
:1013900086E290E0AC01249FC001259F900D349F10
:1013A000900D112490936500809364000FC02091EC
:1013B000640030916500F901E759FF4F8C8180830B
:1013C000C90101969093650080936400EBE2F0E020
:1013D000808188230CF417CE28960FB6F894DEBFD0
:1013E0000FBECDBFCF91DF910895DF93CF93CDB7DF
:1013F000DEB72B970FB6F894DEBF0FBECDBF2BE341
:1014000033E084E59CE0BC01C9010E94700D789432
:10141000A5E5B0E0E5E5F0E0808180648C938895F7
:10142000A5E5B0E0E5E5F0E080818F7B8C93EBE211
:10143000F0E0808188231CF40E94F807E9CF8EE059
:10144000888701C00000488549875985552311F0D8
:1014500081E089878985988591509887882391F7BD
:1014600080916303882309F46BC080916203282F65
:1014700030E086E290E0AC01249FC001259F900DF2
:10148000349F900D112487599F4F9F838E8324E5AD
:1014900030E080916800882F90E0820F931F9D8339
:1014A0008C8386E28887E7E3F0E080EB808325C0C9
:1014B000AFE2B0E0EE81FF818081282F30E0C901EA
:1014C000880F991F820F931F880F991F880F991FEC
:1014D0009C018C819D81820F931F9B838A838E81C7
:1014E0009F8101969F838E83EA81FB81849189830A
:1014F00089818C9300000000000058855A878A85F6
:10150000882311F041E04A878A8598859150988711
:10151000882371F686E0888701C0000058855B87C4
:101520008B85882311F041E04B878B8598859150FE
:101530009887882391F7E7E3F0E080E9808368CF1C
:10154000809160009091610001969093610080937A
:1015500060008091600090916100807098700097A9
:1015600051F08091640090916500FC01E759FF4FB4
:1015700080E280834DCF8091640090916500FC01F2
:10158000E759FF4F8FE7808343CFDF93CF93CDB7EA
:10159000DEB728970FB6F894DEBF0FBECDBF4EC1A1
:1015A000ECE2F0E080818C83809164009091650092
:1015B0008436910509F0B9C084E18B8389E690E017
:1015C0009A838983A0C0E981FA81108289819A81F6
:1015D00001969A838983E981FA81108289819A81AF
:1015E00001969A838983E981FA81108289819A819F
:1015F00001969A838983E981FA81108289819A818F
:1016000001969A838983E981FA81108289819A817E
:1016100001969A838983E981FA81108289819A816E
:1016200001969A838983E981FA81108289819A815E
:1016300001969A838983E981FA81108289819A814E
:1016400001969A838983E981FA81108289819A813E
:1016500001969A838983E981FA81108289819A812E
:1016600001969A838983E981FA81108289819A811E
:1016700001969A838983E981FA81108289819A810E
:1016800001969A838983E981FA81108289819A81FE
:1016900001969A838983E981FA81108289819A81EE
:1016A00001969A838983E981FA81108289819A81DE
:1016B00001969A838983E981FA81108289819A81CE
:1016C00001969A838983E981FA81108289819A81BE
:1016D00001969A838983E981FA81108289819A81AE
:1016E00001969A838983E981FA81108289819A819E
:1016F00001969A838983E981FA81108289819A818E
:1017000001969A8389832B8128873885332311F0AA
:1017100081E0888788859B8191509B83882309F08D
:1017200052CF10926500109264008C81282F30E017
:101730003F832E838E819F818930910569F12E81AF
:101740003F812D30310509F442C08E819F81883060
:10175000910509F064C08091640090916500009744
:1017600009F46CC08091640090916500FC01E75918
:10177000FF4F1082809164009091650001979093D3
:101780006500809364008091640090916500FC0185
:10179000E759FF4F108252C080916400909165001C
:1017A00005968436910508F049C0809164009091B7
:1017B0006500FC01E759FF4F108280916400909111
:1017C00065000596909365008093640037C0809112
:1017D00064009091650025E030E0B9010E94770D2A
:1017E000CB018D838D81833148F580916400909188
:1017F0006500FC01E759FF4F10828D81882F90E032
:101800009C012F5F3F4FC901880F991F880F991FB7
:10181000820F931F90936500809364000FC0209106
:10182000640030916500F901E759FF4F8C81808396
:10183000C90101969093650080936400EBE2F0E0AB
:10184000808188230CF4ACCE28960FB6F894DEBFC6
:101850000FBECDBFCF91DF910895DF93CF93CDB76A
:10186000DEB72D970FB6F894DEBF0FBECDBF7894CC
:10187000A5E5B0E0E5E5F0E0808180648C93889593
:10188000A5E5B0E0E5E5F0E080818F7B8C93EBE2AD
:10189000F0E0808188231CF40E94C50AE9CF809182
:1018A0006303882309F471C080916203282F30E01C
:1018B000C901880F991F880F991F820F931F87599D
:1018C0009F4F9F838E8324E530E08091680086954A
:1018D000882F90E0820F931F9D838C8385E08887FB
:1018E0003BC08FE290E09A878987EE81FF818081FB
:1018F000282F30E0C901880F991F820F931F880F8E
:10190000991F880F991F880F991F9C878B87EB85DC
:10191000FC85FF232CF48B859C8501969C878B8707
:101920008B859C85959587959C018C819D81820FE7
:10193000931F9B838A838E819F8101969F838E83D1
:10194000EA81FB81849189838981E985FA85808395
:10195000E7E3F0E080EB8083F885FD878D858823C1
:1019600011F091E09D878D85988591509887882307
:1019700009F0B7CF000000000000000000000000E8
:10198000E7E3F0E080E9808373CF8091620090917B
:1019900063000196909363008093620080916200DF
:1019A0009091630080709870009751F0809164006E
:1019B00090916500FC01E759FF4F80E2808358CF8A
:1019C0008091640090916500FC01E759FF4F8FE71B
:1019D00080834ECFDF93CF93CDB7DEB70E94030D48
:1019E000E3E3F0E08081882F90E0827090700097B0
:1019F00019F40E94F50902C00E942D0C80E090E0CD
:101A0000CF91DF910895DF93CF93CDB7DEB7A4E3F5
:101A1000B0E0E4E3F0E080818D7F8C93A5E3B0E05B
:101A2000E5E3F0E0808182608C930E94B1070E9420
:101A3000DC07A5E5B0E0E5E5F0E080818F748C93EC
:101A4000E3E3F0E08081882F90E08270907000974F
:101A5000C9F4A4E3B0E0E4E3F0E0808181608C931A
:101A6000EAE4F0E080E094E091838083EEE4F0E04B
:101A700089E08083EFE4F0E01082E9E5F0E080E1C6
:101A800080832BC0A2E3B0E0E2E3F0E080818860D5
:101A90008C93A1E3B0E0E1E3F0E0808188608C9377
:101AA000A2E3B0E0E2E3F0E0808184608C93A1E304
:101AB000B0E0E1E3F0E0808184608C93E3E5F0E066
:101AC0001082E2E5F0E083EC8083E3E5F0E082E081
:101AD0008083E9E5F0E081E08083CF91DF91089594
:101AE000FB01DC0105900D920020E1F70895AA1B8F
:101AF000BB1B51E107C0AA1FBB1FA617B70710F0F9
:101B0000A61BB70B881F991F5A95A9F7809590952A
:0A1B1000BC01CD010895F894FFCF49
:00000001FF
